BL51 BANKED LINKER/LOCATER V6.22                                                        12/03/2024  15:15:46  PAGE 1


BL51 BANKED LINKER/LOCATER V6.22, INVOKED BY:
C:\KEIL_V5\C51\BIN\BL51.EXE .\Objects\STARTUP.obj, .\Objects\main.obj, .\Objects\delay.obj, .\Objects\lcd.obj, .\Objects
>> \rem.obj, .\Objects\key.obj, .\Objects\io.obj TO .\Objects\DM8F52_DEMO PRINT (.\Listings\DM8F52_DEMO.m51) RAMSIZE (25
>> 6)


MEMORY MODEL: SMALL


INPUT MODULES INCLUDED:
  .\Objects\STARTUP.obj (?C_STARTUP)
  .\Objects\main.obj (MAIN)
  .\Objects\delay.obj (DELAY)
  .\Objects\lcd.obj (LCD)
  .\Objects\rem.obj (REM)
  .\Objects\key.obj (KEY)
  .\Objects\io.obj (IO)
  C:\KEIL_V5\C51\LIB\C51S.LIB (?C_INIT)
  C:\KEIL_V5\C51\LIB\C51S.LIB (?C?CLDOPTR)


LINK MAP OF MODULE:  .\Objects\DM8F52_DEMO (?C_STARTUP)


            TYPE    BASE      LENGTH    RELOCATION   SEGMENT NAME
            -----------------------------------------------------

            * * * * * * *   D A T A   M E M O R Y   * * * * * * *
            REG     0000H     0008H     ABSOLUTE     "REG BANK 0"
            DATA    0008H     0008H     UNIT         _DATA_GROUP_
            DATA    0010H     0007H     UNIT         ?DT?REM
            DATA    0017H     0002H     UNIT         ?DT?KEY
            DATA    0019H     0001H     UNIT         ?DT?MAIN
            IDATA   001AH     0001H     UNIT         ?STACK

            * * * * * * *  X D A T A   M E M O R Y  * * * * * * *
            XDATA   0000H     000CH     UNIT         ?XD?REM
                    000CH     FFD4H                  *** GAP ***
            XDATA   FFE0H     001FH     ABSOLUTE     

            * * * * * * *   C O D E   M E M O R Y   * * * * * * *
            CODE    0000H     0003H     ABSOLUTE     
            CODE    0003H     0058H     UNIT         ?PR?REM_DEF?REM
                    005BH     0008H                  *** GAP ***
            CODE    0063H     0003H     ABSOLUTE     
            CODE    0066H     0010H     UNIT         ?PR?MAIN?MAIN
                    0076H     0005H                  *** GAP ***
            CODE    007BH     0003H     ABSOLUTE     
            CODE    007EH     00DEH     UNIT         ?PR?REM_NUM?REM
            CODE    015CH     00D5H     UNIT         ?PR?KEY_SCAN?KEY
            CODE    0231H     008CH     UNIT         ?C_C51STARTUP
            CODE    02BDH     0083H     UNIT         ?PR?REM_INTSETINFRARED?REM
            CODE    0340H     0078H     UNIT         ?PR?LCD_ON?LCD
            CODE    03B8H     0050H     UNIT         ?PR?_INIT_LCD?LCD
            CODE    0408H     0046H     UNIT         ?CO?LCD
            CODE    044EH     003EH     UNIT         ?PR?LCD_ALLOFF?LCD
            CODE    048CH     0035H     UNIT         ?PR?CHANGE_TO_IDLE?MAIN
            CODE    04C1H     0032H     UNIT         ?PR?REM_INIT?REM
BL51 BANKED LINKER/LOCATER V6.22                                                      12/03/2024  15:15:46  PAGE 2


            CODE    04F3H     0030H     UNIT         ?PR?IO_CLR?IO
            CODE    0523H     002DH     UNIT         ?PR?REM_TEST?REM
            CODE    0550H     002DH     UNIT         ?C?LIB_CODE
            CODE    057DH     002AH     UNIT         ?PR?KEY_INIT?KEY
            CODE    05A7H     0028H     UNIT         ?C_INITSEG
            CODE    05CFH     0025H     UNIT         ?PR?REM_HIGH?REM
            CODE    05F4H     0020H     UNIT         ?PR?LCD_OFF?LCD
            CODE    0614H     0016H     UNIT         ?PR?LCD_INIT?LCD
            CODE    062AH     000CH     UNIT         ?PR?SYSTEM_INIT?MAIN
            CODE    0636H     000BH     UNIT         ?PR?_DELAY?DELAY



OVERLAY MAP OF MODULE:   .\Objects\DM8F52_DEMO (?C_STARTUP)


SEGMENT                              DATA_GROUP 
  +--> CALLED SEGMENT              START    LENGTH
--------------------------------------------------
?C_C51STARTUP                      -----    -----
  +--> ?PR?MAIN?MAIN
  +--> ?C_INITSEG

?PR?MAIN?MAIN                      -----    -----
  +--> ?PR?SYSTEM_INIT?MAIN
  +--> ?PR?CHANGE_TO_IDLE?MAIN

?PR?SYSTEM_INIT?MAIN               -----    -----
  +--> ?PR?IO_CLR?IO
  +--> ?PR?LCD_ALLOFF?LCD
  +--> ?PR?KEY_INIT?KEY
  +--> ?PR?CHANGE_TO_IDLE?MAIN

*** NEW ROOT ***************************************************

?PR?REM_INTSETINFRARED?REM         -----    -----
  +--> ?PR?REM_DEF?REM
  +--> ?PR?REM_HIGH?REM

*** NEW ROOT ***************************************************

?PR?KEY_SCAN?KEY                   -----    -----
  +--> ?PR?_DELAY?DELAY
  +--> ?PR?REM_TEST?REM

?PR?REM_TEST?REM                   -----    -----
  +--> ?PR?REM_INIT?REM
  +--> ?PR?LCD_ON?LCD
  +--> ?PR?REM_NUM?REM
  +--> ?PR?LCD_OFF?LCD
  +--> ?PR?REM_HIGH?REM

?PR?LCD_ON?LCD                     -----    -----
  +--> ?PR?LCD_INIT?LCD
  +--> ?CO?LCD

?PR?LCD_INIT?LCD                   -----    -----
BL51 BANKED LINKER/LOCATER V6.22                                                      12/03/2024  15:15:46  PAGE 3


  +--> ?PR?_INIT_LCD?LCD

?PR?_INIT_LCD?LCD                  0008H    0008H

?PR?LCD_OFF?LCD                    -----    -----
  +--> ?PR?LCD_INIT?LCD



SYMBOL TABLE OF MODULE:  .\Objects\DM8F52_DEMO (?C_STARTUP)

  VALUE           TYPE          NAME
  ----------------------------------

  -------         MODULE        ?C_STARTUP
  C:0231H         SEGMENT       ?C_C51STARTUP
  I:001AH         SEGMENT       ?STACK
  C:0000H         PUBLIC        ?C_STARTUP
  D:00E0H         SYMBOL        ACC
  D:00F0H         SYMBOL        B
  D:0083H         SYMBOL        DPH
  D:0082H         SYMBOL        DPL
  N:0000H         SYMBOL        IBPSTACK
  N:0100H         SYMBOL        IBPSTACKTOP
  N:0080H         SYMBOL        IDATALEN
  C:0234H         SYMBOL        IDATALOOP
  N:0000H         SYMBOL        PBPSTACK
  N:0100H         SYMBOL        PBPSTACKTOP
  N:0000H         SYMBOL        PDATALEN
  N:0000H         SYMBOL        PDATASTART
  N:0000H         SYMBOL        PPAGE
  N:0000H         SYMBOL        PPAGEENABLE
  D:00A0H         SYMBOL        PPAGE_SFR
  D:0081H         SYMBOL        SP
  C:0231H         SYMBOL        STARTUP1
  N:0000H         SYMBOL        XBPSTACK
  N:0000H         SYMBOL        XBPSTACKTOP
  N:0000H         SYMBOL        XDATALEN
  N:0000H         SYMBOL        XDATASTART
  C:0000H         LINE#         126
  C:0231H         LINE#         133
  C:0233H         LINE#         134
  C:0234H         LINE#         135
  C:0235H         LINE#         136
  C:0237H         LINE#         185
  C:023AH         LINE#         196
  -------         ENDMOD        ?C_STARTUP

  -------         MODULE        MAIN
  C:0000H         SYMBOL        _ICE_DUMMY_
  C:062AH         PUBLIC        System_Init
  D:0080H         PUBLIC        P0
  D:0090H         PUBLIC        P1
  D:00A0H         PUBLIC        P2
  D:00B0H         PUBLIC        P3
  D:00F5H         PUBLIC        PWM0CON
  D:00C8H         PUBLIC        IEN2
BL51 BANKED LINKER/LOCATER V6.22                                                      12/03/2024  15:15:46  PAGE 4


  D:00D7H         PUBLIC        CLKSTAT
  D:00D4H         PUBLIC        CLKEN0
  D:00D5H         PUBLIC        CLKEN1
  C:0066H         PUBLIC        main
  D:00D3H         PUBLIC        CLKCFG
  D:0087H         PUBLIC        PCON
  D:00D6H         PUBLIC        BORCON
  D:00F1H         PUBLIC        REMCON
  D:00CEH         PUBLIC        WDTCON
  D:0019H         PUBLIC        IDLE_FLG
  D:00D2H         PUBLIC        SYSCON
  D:008AH         PUBLIC        ALFSEL1
  C:048CH         PUBLIC        Change_To_IDLE
  -------         PROC          MAIN
  C:0066H         LINE#         7
  C:0066H         LINE#         8
  C:0066H         LINE#         9
  C:0069H         LINE#         10
  C:0069H         LINE#         11
  C:0069H         LINE#         12
  C:006EH         LINE#         13
  C:006EH         LINE#         14
  C:0071H         LINE#         15
  C:0074H         LINE#         16
  C:0074H         LINE#         17
  -------         ENDPROC       MAIN
  -------         PROC          SYSTEM_INIT
  C:062AH         LINE#         20
  C:062AH         LINE#         21
  C:062AH         LINE#         22
  C:062DH         LINE#         24
  C:0630H         LINE#         25
  C:0633H         LINE#         26
  -------         ENDPROC       SYSTEM_INIT
  -------         PROC          CHANGE_TO_IDLE
  C:048CH         LINE#         29
  C:048CH         LINE#         30
  C:048CH         LINE#         31
  C:048FH         LINE#         32
  C:0492H         LINE#         33
  C:0495H         LINE#         34
  C:0498H         LINE#         36
  C:049BH         LINE#         37
  C:049EH         LINE#         39
  C:04A0H         LINE#         40
  C:04A3H         LINE#         41
  C:04A6H         LINE#         42
  C:04A9H         LINE#         43
  C:04ACH         LINE#         44
  C:04B1H         LINE#         45
  C:04B4H         LINE#         46
  C:04B7H         LINE#         47
  C:04BAH         LINE#         48
  C:04BDH         LINE#         49
  C:04C0H         LINE#         50
  -------         ENDPROC       CHANGE_TO_IDLE
  -------         ENDMOD        MAIN
BL51 BANKED LINKER/LOCATER V6.22                                                      12/03/2024  15:15:46  PAGE 5



  -------         MODULE        DELAY
  C:0000H         SYMBOL        _ICE_DUMMY_
  D:0080H         PUBLIC        P0
  D:0090H         PUBLIC        P1
  D:00A0H         PUBLIC        P2
  D:00B0H         PUBLIC        P3
  C:0636H         PUBLIC        _delay
  -------         PROC          _DELAY
  D:0006H         SYMBOL        n
  C:0636H         LINE#         5
  C:0636H         LINE#         6
  C:0636H         LINE#         7
  C:0640H         LINE#         8
  -------         ENDPROC       _DELAY
  -------         ENDMOD        DELAY

  -------         MODULE        LCD
  C:0000H         SYMBOL        _ICE_DUMMY_
  D:0080H         PUBLIC        P0
  D:0090H         PUBLIC        P1
  D:00A0H         PUBLIC        P2
  D:00B0H         PUBLIC        P3
  C:044EH         PUBLIC        lcd_alloff
  C:0412H         PUBLIC        lcd_num1
  C:0426H         PUBLIC        lcd_num2
  C:043AH         PUBLIC        lcd_num3
  D:00D5H         PUBLIC        CLKEN1
  D:00ABH         PUBLIC        SEGEN1
  D:00ACH         PUBLIC        SEGEN2
  D:00ADH         PUBLIC        SEGEN3
  D:00AEH         PUBLIC        SEGEN4
  D:00AAH         PUBLIC        LCDCON
  C:03B8H         PUBLIC        _init_lcd
  C:05F4H         PUBLIC        lcd_off
  X:FFE0H         PUBLIC        lcd_ram
  D:00D2H         PUBLIC        SYSCON
  C:0408H         PUBLIC        lcd_num
  D:00A9H         PUBLIC        LCDCON1
  C:0614H         PUBLIC        LCD_init
  C:0340H         PUBLIC        lcd_on
  D:00AFH         PUBLIC        COMEN
  -------         PROC          _INIT_LCD
  D:0007H         SYMBOL        vol
  D:0005H         SYMBOL        typesel
  D:0003H         SYMBOL        duty
  D:000BH         SYMBOL        pumpon
  D:000CH         SYMBOL        tlcd
  D:000DH         SYMBOL        fcctl
  D:000EH         SYMBOL        rlcd
  D:000FH         SYMBOL        mod
  C:03B8H         LINE#         11
  C:03B8H         LINE#         19
  C:03B8H         LINE#         20
  C:03BBH         LINE#         21
  C:03BEH         LINE#         23
  C:03C1H         LINE#         24
BL51 BANKED LINKER/LOCATER V6.22                                                      12/03/2024  15:15:46  PAGE 6


  C:03DDH         LINE#         25
  C:03E0H         LINE#         26
  C:03EFH         LINE#         27
  C:03F8H         LINE#         29
  C:03FBH         LINE#         30
  C:03FEH         LINE#         31
  C:0401H         LINE#         32
  C:0404H         LINE#         33
  C:0407H         LINE#         35
  -------         ENDPROC       _INIT_LCD
  -------         PROC          LCD_ON
  -------         DO            
  D:0004H         SYMBOL        unit
  D:0006H         SYMBOL        decade
  -------         ENDDO         
  C:0340H         LINE#         37
  C:0340H         LINE#         38
  C:0340H         LINE#         40
  C:0343H         LINE#         41
  C:0352H         LINE#         42
  C:035FH         LINE#         44
  C:0364H         LINE#         45
  C:0366H         LINE#         46
  C:036AH         LINE#         47
  C:036CH         LINE#         48
  C:037CH         LINE#         49
  C:038CH         LINE#         50
  C:039CH         LINE#         51
  C:03B0H         LINE#         52
  C:03B4H         LINE#         54
  C:03B7H         LINE#         55
  -------         ENDPROC       LCD_ON
  -------         PROC          LCD_OFF
  C:05F4H         LINE#         57
  C:05F4H         LINE#         58
  C:05F4H         LINE#         59
  C:05F7H         LINE#         60
  C:05FCH         LINE#         61
  C:05FEH         LINE#         62
  C:0602H         LINE#         63
  C:0604H         LINE#         64
  C:0606H         LINE#         65
  C:0608H         LINE#         66
  C:060AH         LINE#         67
  C:060CH         LINE#         68
  C:0610H         LINE#         69
  C:0613H         LINE#         70
  -------         ENDPROC       LCD_OFF
  -------         PROC          LCD_ALLOFF
  C:044EH         LINE#         71
  C:044EH         LINE#         72
  C:044EH         LINE#         73
  C:0451H         LINE#         74
  C:0454H         LINE#         76
  C:0457H         LINE#         77
  C:045AH         LINE#         78
  C:045CH         LINE#         79
BL51 BANKED LINKER/LOCATER V6.22                                                      12/03/2024  15:15:46  PAGE 7


  C:045FH         LINE#         80
  C:0462H         LINE#         82
  C:0464H         LINE#         83
  C:0467H         LINE#         84
  C:046AH         LINE#         85
  C:046DH         LINE#         86
  C:0470H         LINE#         87
  C:0474H         LINE#         88
  C:0476H         LINE#         89
  C:047AH         LINE#         90
  C:047CH         LINE#         91
  C:047EH         LINE#         92
  C:0480H         LINE#         93
  C:0482H         LINE#         94
  C:0484H         LINE#         95
  C:0488H         LINE#         96
  C:048BH         LINE#         97
  -------         ENDPROC       LCD_ALLOFF
  -------         PROC          LCD_INIT
  C:0614H         LINE#         99
  C:0614H         LINE#         100
  C:0614H         LINE#         102
  -------         ENDPROC       LCD_INIT
  -------         ENDMOD        LCD

  -------         MODULE        REM
  C:0000H         SYMBOL        _ICE_DUMMY_
  D:0080H         PUBLIC        P0
  D:0090H         PUBLIC        P1
  D:00A0H         PUBLIC        P2
  D:00B0H         PUBLIC        P3
  D:00B7H         PUBLIC        P5
  B:00A8H.7       PUBLIC        EA
  D:00F5H         PUBLIC        PWM0CON
  X:0000H         PUBLIC        OFF_R
  D:00C8H         PUBLIC        IEN2
  C:007EH         PUBLIC        REM_num
  D:00D7H         PUBLIC        CLKSTAT
  D:00E6H         PUBLIC        P5CR
  D:00F2H         PUBLIC        REMNUMH
  D:00D4H         PUBLIC        CLKEN0
  D:00D5H         PUBLIC        CLKEN1
  D:00F3H         PUBLIC        REMNUML
  D:00D3H         PUBLIC        CLKCFG
  D:00F1H         PUBLIC        REMCON
  D:0010H         PUBLIC        ADD
  X:0006H         PUBLIC        ON_R
  C:02BDH         PUBLIC        REM_IntSetInfrared
  D:0013H         PUBLIC        bz
  C:04C1H         PUBLIC        rem_init
  D:00D2H         PUBLIC        SYSCON
  C:05CFH         PUBLIC        REM_high
  C:0523H         PUBLIC        REM_Test
  D:0014H         PUBLIC        i
  D:0015H         PUBLIC        j
  D:00F7H         PUBLIC        PWM0D
  D:0016H         PUBLIC        k
BL51 BANKED LINKER/LOCATER V6.22                                                      12/03/2024  15:15:46  PAGE 8


  D:008AH         PUBLIC        ALFSEL1
  D:00D1H         PUBLIC        CKCON
  C:0003H         PUBLIC        REM_def
  D:00F6H         PUBLIC        PWM0P
  -------         PROC          REM_INIT
  C:04C1H         LINE#         16
  C:04C1H         LINE#         17
  C:04C1H         LINE#         18
  C:04C4H         LINE#         19
  C:04C7H         LINE#         20
  C:04CAH         LINE#         21
  C:04CDH         LINE#         22
  C:04D0H         LINE#         23
  C:04D3H         LINE#         24
  C:04D8H         LINE#         25
  C:04DBH         LINE#         26
  C:04DEH         LINE#         27
  C:04E1H         LINE#         28
  C:04E4H         LINE#         29
  C:04E6H         LINE#         31
  C:04E9H         LINE#         32
  C:04ECH         LINE#         33
  C:04EFH         LINE#         34
  C:04F2H         LINE#         37
  -------         ENDPROC       REM_INIT
  -------         PROC          REM_TEST
  C:0523H         LINE#         39
  C:0523H         LINE#         40
  C:0523H         LINE#         41
  C:0526H         LINE#         42
  C:0529H         LINE#         43
  C:0530H         LINE#         44
  C:0530H         LINE#         45
  C:0530H         LINE#         46
  C:0533H         LINE#         47
  C:0536H         LINE#         48
  C:053FH         LINE#         49
  C:0541H         LINE#         50
  C:0541H         LINE#         51
  C:0544H         LINE#         52
  C:054DH         LINE#         53
  C:054DH         LINE#         54
  C:054DH         LINE#         55
  C:054DH         LINE#         56
  C:054DH         LINE#         57
  -------         ENDPROC       REM_TEST
  -------         PROC          REM_NUM
  C:007EH         LINE#         60
  C:007EH         LINE#         61
  C:007EH         LINE#         62
  C:00C2H         LINE#         63
  C:00C2H         LINE#         64
  C:00C2H         LINE#         65
  C:00C8H         LINE#         66
  C:00CCH         LINE#         67
  C:00CDH         LINE#         68
  C:00CDH         LINE#         69
BL51 BANKED LINKER/LOCATER V6.22                                                      12/03/2024  15:15:46  PAGE 9


  C:00D3H         LINE#         70
  C:00D7H         LINE#         71
  C:00D8H         LINE#         72
  C:00D8H         LINE#         73
  C:00DEH         LINE#         74
  C:00E2H         LINE#         75
  C:00E3H         LINE#         76
  C:00E3H         LINE#         77
  C:00E9H         LINE#         78
  C:00EDH         LINE#         79
  C:00EEH         LINE#         80
  C:00EEH         LINE#         81
  C:00F4H         LINE#         82
  C:00F8H         LINE#         83
  C:00F9H         LINE#         84
  C:00F9H         LINE#         85
  C:00FFH         LINE#         86
  C:0103H         LINE#         87
  C:0104H         LINE#         88
  C:0104H         LINE#         89
  C:010AH         LINE#         90
  C:010EH         LINE#         91
  C:010FH         LINE#         92
  C:010FH         LINE#         93
  C:0115H         LINE#         94
  C:0119H         LINE#         95
  C:011AH         LINE#         96
  C:011AH         LINE#         97
  C:0120H         LINE#         98
  C:0124H         LINE#         99
  C:0125H         LINE#         100
  C:0125H         LINE#         101
  C:012BH         LINE#         102
  C:012FH         LINE#         103
  C:0130H         LINE#         104
  C:0130H         LINE#         105
  C:0136H         LINE#         106
  C:013AH         LINE#         107
  C:013BH         LINE#         108
  C:013BH         LINE#         109
  C:0141H         LINE#         110
  C:0145H         LINE#         111
  C:0146H         LINE#         112
  C:0146H         LINE#         113
  C:014CH         LINE#         114
  C:0150H         LINE#         115
  C:0151H         LINE#         116
  C:0151H         LINE#         117
  C:0157H         LINE#         118
  C:015BH         LINE#         119
  C:015BH         LINE#         120
  C:015BH         LINE#         121
  C:015BH         LINE#         122
  C:015BH         LINE#         123
  -------         ENDPROC       REM_NUM
  -------         PROC          REM_HIGH
  C:05CFH         LINE#         126
BL51 BANKED LINKER/LOCATER V6.22                                                      12/03/2024  15:15:46  PAGE 10


  C:05CFH         LINE#         127
  C:05CFH         LINE#         128
  C:05D6H         LINE#         129
  C:05DDH         LINE#         130
  C:05DDH         LINE#         131
  C:05E0H         LINE#         132
  C:05E3H         LINE#         133
  C:05E6H         LINE#         134
  C:05E7H         LINE#         136
  C:05E7H         LINE#         137
  C:05EAH         LINE#         138
  C:05EDH         LINE#         139
  C:05F0H         LINE#         140
  C:05F3H         LINE#         141
  C:05F3H         LINE#         144
  -------         ENDPROC       REM_HIGH
  -------         PROC          REM_DEF
  C:0003H         LINE#         146
  C:0003H         LINE#         147
  C:0003H         LINE#         149
  C:000DH         LINE#         150
  C:000DH         LINE#         151
  C:0011H         LINE#         153
  C:0011H         LINE#         154
  C:003DH         LINE#         155
  C:003DH         LINE#         156
  C:0040H         LINE#         157
  C:0042H         LINE#         158
  C:0044H         LINE#         160
  C:0044H         LINE#         161
  C:0047H         LINE#         162
  C:0049H         LINE#         163
  C:0049H         LINE#         164
  C:0055H         LINE#         165
  C:0055H         LINE#         166
  C:0058H         LINE#         167
  C:005AH         LINE#         168
  C:005AH         LINE#         170
  -------         ENDPROC       REM_DEF
  -------         PROC          REM_INTSETINFRARED
  C:02BDH         LINE#         173
  C:02D8H         LINE#         177
  C:02F1H         LINE#         178
  C:02F1H         LINE#         179
  C:02F1H         LINE#         180
  C:02F4H         LINE#         181
  C:02F7H         LINE#         182
  C:02F7H         LINE#         183
  C:02F9H         LINE#         184
  C:02F9H         LINE#         185
  C:02FCH         LINE#         186
  C:02FFH         LINE#         187
  C:0302H         LINE#         188
  C:0304H         LINE#         189
  C:0304H         LINE#         190
  C:0307H         LINE#         191
  C:030AH         LINE#         192
BL51 BANKED LINKER/LOCATER V6.22                                                      12/03/2024  15:15:46  PAGE 11


  C:030AH         LINE#         193
  C:030CH         LINE#         194
  C:030CH         LINE#         195
  C:030FH         LINE#         196
  C:0312H         LINE#         197
  C:0315H         LINE#         198
  C:0317H         LINE#         199
  C:0317H         LINE#         200
  C:0319H         LINE#         201
  C:031CH         LINE#         202
  C:031EH         LINE#         203
  C:031EH         LINE#         204
  C:0321H         LINE#         205
  C:0324H         LINE#         206
  C:0327H         LINE#         207
  C:0327H         LINE#         208
  C:0327H         LINE#         209
  C:0327H         LINE#         210
  C:0327H         LINE#         213
  -------         ENDPROC       REM_INTSETINFRARED
  -------         ENDMOD        REM

  -------         MODULE        KEY
  C:0000H         SYMBOL        _ICE_DUMMY_
  D:0080H         PUBLIC        P0
  D:00B1H         PUBLIC        INTEN
  D:0090H         PUBLIC        P1
  D:00A0H         PUBLIC        P2
  D:00B0H         PUBLIC        P3
  B:00A8H.7       PUBLIC        EA
  D:00C8H         PUBLIC        IEN2
  D:00E2H         PUBLIC        P1CR
  D:00B2H         PUBLIC        INTCTRL
  D:0017H         PUBLIC        TEMP
  D:00B3H         PUBLIC        INTFLG
  C:015CH         PUBLIC        KEY_Scan
  C:057DH         PUBLIC        key_init
  D:00EAH         PUBLIC        P1PCR
  D:0018H         PUBLIC        KEY
  -------         PROC          KEY_INIT
  C:057DH         LINE#         7
  C:057DH         LINE#         8
  C:057DH         LINE#         9
  C:0583H         LINE#         10
  C:0589H         LINE#         11
  C:058FH         LINE#         12
  C:0595H         LINE#         13
  C:0597H         LINE#         14
  C:059AH         LINE#         15
  C:059DH         LINE#         16
  C:05A0H         LINE#         18
  C:05A3H         LINE#         19
  C:05A6H         LINE#         20
  -------         ENDPROC       KEY_INIT
  -------         PROC          KEY_SCAN
  C:015CH         LINE#         23
  C:0179H         LINE#         26
BL51 BANKED LINKER/LOCATER V6.22                                                      12/03/2024  15:15:46  PAGE 12


  C:018FH         LINE#         27
  C:018FH         LINE#         28
  C:018FH         LINE#         29
  C:0192H         LINE#         30
  C:0195H         LINE#         31
  C:019CH         LINE#         32
  C:01A5H         LINE#         33
  C:01A5H         LINE#         34
  C:01A8H         LINE#         35
  C:01A8H         LINE#         36
  C:01AAH         LINE#         40
  C:01AAH         LINE#         41
  C:01ADH         LINE#         42
  C:01B0H         LINE#         43
  C:01B7H         LINE#         44
  C:01C0H         LINE#         45
  C:01C0H         LINE#         46
  C:01C3H         LINE#         47
  C:01C3H         LINE#         48
  C:01C5H         LINE#         50
  C:01C5H         LINE#         51
  C:01C7H         LINE#         52
  C:01C7H         LINE#         53
  C:01CAH         LINE#         54
  C:01CDH         LINE#         55
  C:01D4H         LINE#         56
  C:01E4H         LINE#         57
  C:01E4H         LINE#         58
  C:01E6H         LINE#         59
  C:01E6H         LINE#         60
  C:01E8H         LINE#         62
  C:01E8H         LINE#         63
  C:01EAH         LINE#         64
  C:01EAH         LINE#         65
  C:01EDH         LINE#         66
  C:01F0H         LINE#         67
  C:01F7H         LINE#         68
  C:0207H         LINE#         69
  C:0207H         LINE#         70
  C:0209H         LINE#         71
  C:020CH         LINE#         72
  C:020EH         LINE#         74
  C:020EH         LINE#         75
  C:0210H         LINE#         76
  C:0210H         LINE#         77
  C:0213H         LINE#         78
  C:0216H         LINE#         79
  C:0216H         LINE#         80
  C:0216H         LINE#         82
  -------         ENDPROC       KEY_SCAN
  -------         ENDMOD        KEY

  -------         MODULE        IO
  C:0000H         SYMBOL        _ICE_DUMMY_
  D:0080H         PUBLIC        P0
  D:0090H         PUBLIC        P1
  D:00A0H         PUBLIC        P2
BL51 BANKED LINKER/LOCATER V6.22                                                      12/03/2024  15:15:46  PAGE 13


  D:00B0H         PUBLIC        P3
  D:00BFH         PUBLIC        P4
  D:00B7H         PUBLIC        P5
  D:00E1H         PUBLIC        P0CR
  D:00E2H         PUBLIC        P1CR
  D:00E3H         PUBLIC        P2CR
  D:00E4H         PUBLIC        P3CR
  D:00E5H         PUBLIC        P4CR
  D:00E6H         PUBLIC        P5CR
  C:04F3H         PUBLIC        IO_CLR
  D:00E9H         PUBLIC        P0PCR
  D:00EAH         PUBLIC        P1PCR
  D:00EBH         PUBLIC        P2PCR
  D:0089H         PUBLIC        ALFSEL0
  D:00ECH         PUBLIC        P3PCR
  D:008AH         PUBLIC        ALFSEL1
  D:00EDH         PUBLIC        P4PCR
  D:00EEH         PUBLIC        P5PCR
  -------         PROC          IO_CLR
  C:04F3H         LINE#         6
  C:04F3H         LINE#         7
  C:04F3H         LINE#         8
  C:04F6H         LINE#         9
  C:04F9H         LINE#         10
  C:04FCH         LINE#         11
  C:04FFH         LINE#         12
  C:0502H         LINE#         13
  C:0505H         LINE#         15
  C:0508H         LINE#         16
  C:050BH         LINE#         17
  C:050DH         LINE#         18
  C:050FH         LINE#         19
  C:0511H         LINE#         20
  C:0513H         LINE#         22
  C:0515H         LINE#         23
  C:0517H         LINE#         25
  C:0519H         LINE#         26
  C:051BH         LINE#         27
  C:051DH         LINE#         28
  C:051FH         LINE#         29
  C:0522H         LINE#         30
  -------         ENDPROC       IO_CLR
  -------         ENDMOD        IO

  -------         MODULE        ?C?CLDOPTR
  C:0550H         PUBLIC        ?C?CLDOPTR
  -------         ENDMOD        ?C?CLDOPTR

Program Size: data=27.0 xdata=43 code=1588
LINK/LOCATE RUN COMPLETE.  0 WARNING(S),  0 ERROR(S)
